:020000020000FC
:10780000F8940FE50DBF08E00EBF08E101BD077F4A
:1078100001BD8898909A02E0A3E0B0E01197F1F7DB
:10782000809B1DC00A95C1F7819BFECF90980027D1
:107830000093E40000E000BD00E109B908E00AB9E6
:10784000002700936200E6E2FEE79CD18CD1009114
:10785000E4000023D9F700270AB90C9400000027A0
:10786000009325010093E400009360000093610001
:1078700000E000BD00E109B908E10AB900E80093A1
:1078800062000FEF0093E300222433244424ECEE43
:10789000FCE778D168D10091600005FF03C0E0EB00
:1078A000FEE770D104FDACCF00916100002309F424
:1078B000F1CFE5E2F1E01191123038F001910A3395
:1078C00009F405C0ECE3FEE75DD15CD0E3CF1B30EB
:1078D000C8F33327D8D0B0F3202FD5D098F3D02FCA
:1078E000D2D080F3C02FCFD068F31950003019F0F8
:1078F0000130B1F0EACF222349F0C5D018F3D037D8
:1079000008F03AC047D198F12A95A9F70FEF302730
:1079100033953F93B8D03F91A8F2301719F51EC0A8
:10792000222381F60FEF302733953F93ACD03F9160
:1079300008F4C8CF3017B1F46CD1C8F0032D89D04A
:10794000022D87D0E0EEFEE71DD1042D82D0EEEFB0
:10795000FEE718D122243324442400C0E0E6FEE7E9
:1079600011D1B3CFEEE9FEE70DD14394AECFE4E6FB
:10797000FEE708D14394A9CFE8E7FEE703D143949B
:10798000A4CFFFCF0F931F932F93CF93DF93EF934A
:10799000FF9322270027E6E2F1E0C5E2D1E019914A
:1079A000112391F009910D3031F01A95D9F705C0E6
:1079B0000991019323951A95D9F7209325010091F8
:1079C0006100002319F00A9500936100FF91EF9187
:1079D000DF91CF912F911F910F9108950F931F93D6
:1079E000CF93DF931BB10CB114FD23C013FD27C04F
:1079F0000D3021F0003240F10F3730F5C5E2D1E013
:107A000018811F3708F55FD0013618F00B3708F4DE
:107A1000005213951883C10F1127D11F08830D3011
:107A200099F40AE050D00091610003950093610041
:107A30000BC00091600000610093600005C00091E0
:107A40006000006200936000DF91CF911F910F9161
:107A500008950F931F930F93069506950695069527
:107A600010E3010F0A3310F017E0010F2CD00F9133
:107A70000F7010E3010F0A3310F017E0010F23D04D
:107A80001F910F9108951F9301910033C8F0005387
:107A90000A3028F00131A0F0073190F40750029528
:107AA0001191103368F010531A3028F0113140F062
:107AB000173130F41750012B300F88941F9108951F
:107AC00008941F9108951F932F93CF93DF931091E4
:107AD000E4001F3310F047D0FACFC4EED0E0188195
:107AE00013951883C10F2227D21F088320916000AD
:107AF000226020936000113009F40CB910916200EB
:107B0000106210936200DF91CF912F911F91089521
:107B10000F931F93CF93DF93C4EED0E0088100232F
:107B200019F00A95099331F4009160000D7F0093DC
:107B300060000FC0CF93DF93198119930A95E1F785
:107B4000DF91CF9108810CB9DF91CF911F910F91F7
:107B50000895009162000F7D00936200DF91CF9144
:107B60001F910F9108950F930091620007FF02C0CB
:107B70005F9934DF0091620005FF02C05D99C8DFA4
:107B80000F9108950F930591002311F09CDFFBCF17
:107B90000F9108951F93EF93FF93239429F4339447
:107BA00019F41FEF212E312ECF93DF93FF91EF9128
:107BB0001127F695E7950894111F1034D0F3109112
:107BC000E3001F3FC1F01E1799F4E093E300CF9349
:107BD000DF93CF77DD2713E6C10F10E0D11F0883B5
:107BE000DF91CF912196FF91EF911F918894089595
:107BF00010D008F409C0EF93CF93DF93FF91EF917A
:107C0000E07820D0EF91E1CFFF91EF911F910894A0
:107C100008950F931F93EF93FF931091E300EE27C6
:107C2000FF27112331F000E8E00F0027F01F1A951D
:107C3000D1F70FEF0093E30016D0FF91EF911F9162
:107C40000F9108950F93AF93BF93EF93FF93A3E624
:107C5000B0E005910D93A33EE1F7FF91EF91BF9145
:107C6000AF910F9108950F931F93AF93BF930F920E
:107C70001F9203E02CD001E12AD0EF93FF93A3E6FB
:107C8000B0E010E80D901D9001E021D03296125026
:107C9000C9F7FF91EF9105E01AD001E118D0EF93F9
:107CA000FF93A3E6B0E005911D91011761F4A33E97
:107CB000D1F7FF91EF9188941F900F90BF91AF91F2
:107CC0001F910F910895FF91EF910894F5CF1F93A5
:107CD0004ADF17B710FDFCCF1FB7F89444DFE199D6
:107CE000FDCF07BFE8951FBF1F9108950D0A202003
:107CF00020202020202020602E2D2E20202020201B
:107D00002E2D2E600D0A202020202020605C2E2D9C
:107D10002D2E205C2E5E2E2F202E2D2D2E2F60201E
:107D20000D0A2020202020202020202C20205C2F25
:107D30006020605C2F20202C0D0A20202020202095
:107D400020202F20605C7C20202020207C2F6020A1
:107D50005C200D0A202020202020202F2020202001
:107D60007C602D2D2D277C202020205C0D0A2020DA
:107D700020202E2D27202C2D27607C202020202025
:107D80007C60272D2C20272D2E200D0A202020203E
:107D9000202020207C2020207C2020205C207C2093
:107DA00020207C200D0A20202020202020207C2044
:107DB00020205C202020202C2F2020207C200D0A39
:107DC000202020202020202E2720202020602D5F12
:107DD0002D2720202020202E0D0A436F636B726F09
:107DE00061636849492076302E3032200D0A53698C
:107DF0006D6F6E20536368696573736C20287369B7
:107E00006D6F6E5F7340616C756D2E6D69742E655C
:107E1000647529200D0A426F6F746C6F6164206D68
:107E20006F64650D0A00457865637574652070722E
:107E30006F6772616D2E2E2E0D0A000053796E74DD
:107E40006178206572726F720D0A00005061727362
:107E5000696E67206865782D6C696E650D0A000093
:107E60002A0D0A00466C6173682077726974652078
:107E70006572726F720D0A0044617461206D7573D2
:107E800074206E6F7420626520696E20626F6F745B
:107E90006C6F61642061726561210D0A00004368A6
:107EA00065636B73756D206572726F720D0A0000E9
:107EB00052656365697665206572726F7221205321
:107EC0006574206C696E652064656C617920746FDF
:107ED00020356D73206F72206D6F72652E0D0A0054
:107EE000206279746573207772697474656E20748A
:107EF0006F20464C41534820776974682000206504
:0A7F000072726F72732E0D0A0000FA
:00000001FF
